:100000000C9462000C948A000C948A000C948A0070
:100010000C948A000C948A000C948A000C948A0038
:100020000C948A000C948A000C948A000C948A0028
:100030000C948A000C948A000C948A000C948A0018
:100040000C94EA000C948A000C945C020C948A00D4
:100050000C948A000C948A000C948A000C948A00F8
:100060000C948A000C948A000000000024002700F1
:100070002A0000000000250028002B0000000000DE
:1000800023002600290004040404040404040202DA
:100090000202020203030303030301020408102007
:1000A0004080010204081020010204081020000012
:1000B0000007000201000003040600000000000029
:1000C0000000A50311241FBECFEFD4E0DEBFCDBFDB
:1000D00011E0A0E0B1E0E2E4F9E002C005900D9289
:1000E000AE30B107D9F711E0AEE0B1E001C01D922A
:1000F000AE3AB107E1F710E0C4ECD0E004C02297BB
:10010000FE010E949B04C23CD107C9F70E94E30094
:100110000C949F040C9400001092030110920201B1
:1001200013C0809100010E94960165E070E080E0BC
:1001300090E00E94320180910201909103010196AA
:100140009093030180930201609102017091030179
:100150006F3F710531F32CF38EEF90E00FC080916B
:1001600000010E9496016AE070E080E090E00E9449
:100170003201809102019091030101979093030154
:1001800080930201609102017091030177FFE7CF34
:1001900068EC70E080E090E00E94320108958BE905
:1001A00091E040E855E260E070E00E9499028091A1
:1001B000000161E00E94EF018091000160E070E0C9
:1001C0000E94960108950E945C010E94CF000E9447
:1001D0008C00FDCF1F920F920FB60F9211242F9318
:1001E0003F938F939F93AF93BF9380911201909110
:1001F0001301A0911401B0911501309116010196DF
:10020000A11DB11D232F2D5F2D3720F02D570196F5
:10021000A11DB11D2093160180931201909313012B
:10022000A0931401B093150180910E0190910F01DC
:10023000A0911001B09111010196A11DB11D8093F3
:100240000E0190930F01A0931001B0931101BF9183
:10025000AF919F918F913F912F910F900FBE0F9073
:100260001F901895EF92FF920F931F937B018C01C3
:100270008FB7F894409112015091130160911401CD
:10028000709115018FBF2FB7F89480911201909152
:100290001301A0911401B09115012FBF841B950B80
:1002A000A60BB70BE816F9060A071B0760F71F91A4
:1002B0000F91FF90EF900895789484B5826084BD8B
:1002C00084B5816084BD85B5826085BD85B581605A
:1002D00085BDEEE6F0E0808181608083E1E8F0E0BA
:1002E000808182608083808181608083E0E8F0E0AB
:1002F000808181608083E1EBF0E080818460808395
:10030000E0EBF0E0808181608083EAE7F0E08081CB
:10031000846080838081826080838081816080832B
:100320008081806880831092C10008951F93CF93CD
:10033000DF93182FEB0161E00E94EF01E12FF0E065
:10034000E255FF4F8491833051F4809180008068A2
:1003500080938000D0938900C09388003CC0843093
:1003600051F480918000806280938000D0938B0054
:10037000C0938A0030C0813039F4209729F184B5C8
:10038000806884BDC7BD27C0823039F42097E1F072
:1003900084B5806284BDC8BD1EC0863041F48091A2
:1003A000B00080688093B000C093B30014C0873061
:1003B00041F48091B00080628093B000C093B4009B
:1003C0000AC0C038D1051CF4812F60E002C0812F23
:1003D00061E00E940F02DF91CF911F910895282FB5
:1003E00030E0C90186569F4FFC0194912A573F4F38
:1003F000F9018491882391F0E82FF0E0EE0FFF1FC0
:10040000E859FF4FA591B491662329F48C919095FA
:1004100089238C9308958C91892B8C930895482F70
:1004200050E0CA0182559F4FFC012491CA018656B3
:100430009F4FFC0194914A575F4FFA013491332347
:10044000D1F1222331F1233021F4809180008F7784
:1004500005C0243031F4809180008F7D809380002E
:1004600018C0213019F484B58F7704C0223021F4EC
:1004700084B58F7D84BD0DC0263021F48091B000FD
:100480008F7705C0273029F48091B0008F7D80934D
:10049000B000E32FF0E0EE0FFF1FEE58FF4FA591E5
:1004A000B491662329F48C91909589238C930895B7
:1004B0008C91892B8C9308951F920F920FB60F92F7
:1004C00011242F933F934F935F936F937F938F9359
:1004D0009F93AF93BF93EF93FF934091C600E0913A
:1004E0009701F0919801CF01019660E870E00E94B9
:1004F00035049C018091990190919A012817390740
:1005000039F0E95EFE4F40833093980120939701C4
:10051000FF91EF91BF91AF919F918F917F916F91DB
:100520005F914F913F912F910F900FBE0F901F90B1
:1005300018955F926F927F928F929F92AF92BF9227
:10054000CF92DF92EF92FF920F931F93CF93DF939F
:10055000EC013A014B01413482E458078FE068070F
:1005600080E078070CF07FC060E874E88EE190E0EE
:10057000A40193010E946A04215030404040504041
:10058000CA01B90122E030E040E050E00E946A0474
:1005900059016A01A6019501209530954095509525
:1005A00094E0220F331F441F551F9A95D1F760E046
:1005B00074E284EF90E00E946A04CA01B9012FEF4F
:1005C00030E040E050E00E941604A40193010E9434
:1005D0006A04C90181509F4F181619061CF4522E47
:1005E0005A9403C055245394521A60E079E08DE385
:1005F00090E0A40193010E946A04215030404040E1
:100600005040CA01B90122E030E040E050E00E94D1
:100610006A04209530954095509583E0220F331F52
:10062000441F551F8A95D1F760E074E284EF90E093
:100630000E946A04CA01B9012FEF30E040E050E0A7
:100640000E941604A40193010E946A04C90181500A
:100650009F4F181619061CF4822F815002C081E0AA
:10066000821B851500F5E885F98581E090E00A8810
:1006700002C0880F991F0A94E2F7808360E079E056
:100680008DE390E0A40193010E946A042150304060
:1006900040405040CA01B90122E030E040E050E063
:1006A0000E946A0404C0E885F98510829501EC81F6
:1006B000FD813083EE81FF812083EA85FB852081E7
:1006C00041E050E0CA010E8402C0880F991F0A94CD
:1006D000E2F7282B2083EA85FB852081CA010F845D
:1006E00002C0880F991F0A94E2F7282B2083EA851D
:1006F000FB858081088802C0440F551F0A94E2F7E9
:10070000842B8083DF91CF911F910F91FF90EF9009
:10071000DF90CF90BF90AF909F908F907F906F9021
:100720005F900895FC01A085B18521898C9190E0AE
:10073000022E02C0959587950A94E2F780FFF6CFC6
:100740000484F585E02D6083089588E091E090931E
:100750009C0180939B0187E191E090939E0180939F
:100760009D0185EC90E09093A00180939F0184EC23
:1007700090E09093A2018093A10180EC90E090938F
:10078000A4018093A30181EC90E09093A601809353
:10079000A50186EC90E09093A8018093A70184E0E6
:1007A0008093A90183E08093AA0187E08093AB0145
:1007B00085E08093AC0181E08093AD0108950F93B3
:1007C0001F93CF93DF938C01EB0109C02196D801D1
:1007D000ED91FC910190F081E02DC80109956881AF
:1007E0006623A1F7DF91CF911F910F910895EF92AA
:1007F000FF920F931F93CF93DF938C017B01EA014C
:100800000CC0D7016D917D01D801ED91FC91019053
:10081000F081E02DC80109952197209791F7DF918C
:10082000CF911F910F91FF90EF900895629FD0019B
:10083000739FF001829FE00DF11D649FE00DF11D9B
:10084000929FF00D839FF00D749FF00D659FF00D4A
:100850009927729FB00DE11DF91F639FB00DE11D37
:10086000F91FBD01CF011124089597FB092E07261A
:100870000AD077FD04D049D006D000201AF4709534
:1008800061957F4F0895F6F7909581959F4F089554
:10089000A1E21A2EAA1BBB1BFD010DC0AA1FBB1F84
:1008A000EE1FFF1FA217B307E407F50720F0A21BF6
:1008B000B30BE40BF50B661F771F881F991F1A9463
:1008C00069F760957095809590959B01AC01BD018D
:1008D000CF01089597FB092E05260ED057FD04D0B1
:1008E000D7DF0AD0001C38F45095409530952195FB
:1008F0003F4F4F4F5F4F0895F6F790958095709555
:1009000061957F4F8F4F9F4F0895AA1BBB1B51E1ED
:1009100007C0AA1FBB1FA617B70710F0A61BB70B6F
:10092000881F991F5A95A9F780959095BC01CD0114
:100930000895EE0FFF1F0590F491E02D0994F894AF
:02094000FFCFE7
:0E0942000B000100000000009203DF03F7032A
:00000001FF
